:100EB8001201000200000040051603800100010233
:100EC80000010A060002000000400100090220009B
:100ED800010100A0FA0904000002FF000000070554
:100EE8000202000200070586020002000902200033
:100EF800010100A0FA0904000002FF000000070534
:100F08000102400000070581024000001203410071
:100F180042004300440045004600470048002603BD
:100F280041004300430045005300200049002F00C2
:100F38004F002000500072006F00640075006300CD
:100F4800740073001E035500530042002D00440036
:100F580049004F002D003900360000000000000055
:040F68000000000085
:101B7F005553422D44494F2D3438005553422D446F
:101B8F00494F2D3936004143434553205553422D7C
:011B9F000045
:0400460043B1202280
:04004E0053B1DF22A9
:041DD30063B12022B6
:10174B00EF5407FE7401A806088002C333D8FCFED1
:10175B00EF131313540FFFD3940540020F0FED60DB
:10176B000EE42FF582E43480F583E04EF08011E433
:10177B002FF582E43480F583E0FFEEF4FEEF5EF0AC
:03178B00021DD369
:101A1400EF131313541FFEE42EF582E43480F58390
:101A2400E0FEEF5407FF7401A807088002C333D80F
:0C1A3400FC5206EE60047F0180027F007F
:011A40002283
:10122500908000E0120D39908001E0900001120DD0
:101235004B908002E0900002120D4B908003E090ED
:101245000003120D4B908004E0900004120D4B90AA
:101255008005E0900005120D4B30093C908008E0B8
:10126500900006120D4B908009E0900007120D4B7F
:1012750090800AE0900008120D4B90800BE09000E2
:1012850009120D4B90800CE090000A120D4B9080D6
:091295000DE090000B120D4B223C
:061436008B328A33893479
:10143C00E4FFAB32AA33A9348F82758300120D0CF2
:10144C00FE74FB2FF582E43428F583EEF0E42FF5DF
:10145C0082E43480F583EEF0300925EF2406F58222
:10146C00E433F583120D0CFE74012FF582E434295C
:10147C00F583EEF074082FF582E43480F583EEF0FA
:04148C000FBF06AEDA
:011490002239
:101AC500E4FF74FB2FF582E43428F58374FFF0748A
:101AD500012FF582E43429F58374FFF00FBF06E288
:0A1AE5009028F974FFF0A3740FF0CD
:011AEF0022D4
:1014910090E600E054E7F07580FF75900F75B2FF9C
:1014A10075B31F75B6209028F9E0F580A3E0540FBD
:1014B100F590E4FF74FB2FF582E43428F583E0FE18
:1014C100E42FF582E43480F583EEF03009187401DD
:1014D1002FF582E43429F583E0FE74082FF582E4C8
:0A14E1003480F583EEF00FBF06CA59
:0114EB0022DE
:1011A500EF131313541FFEED131313541FFC5307B2
:1011B5000753050774902EF582E43428F583E0FB88
:1011C5007A0074017E00A807088005C333CE33CEAC
:1011D500D8F9FFEE5AFEEF5B4E6003D38001C39250
:1011E50005300402B20530051A74902CF582E434FA
:1011F50028F583E0FF7401A805088002C333D8FCF5
:101205004FF02274902CF582E43428F583E0FFAE8C
:0F121500057401A806088002C333D8FCF45FF00B
:0112240022A7
:1017CD00E4FFE42FF582E43480F583E0FE74902F7E
:1017DD00F582E43428F583EEF030091874082FF5FE
:1017ED0082E43480F583E0FE74962FF582E434288C
:0817FD00F583EEF00FBF06CAF0
:0118050022C0
:10180600E4FF74902FF582E43428F583E0FEE42F9C
:10181600F582E43480F583EEF030091874962FF5DE
:1018260082E43428F583E0FE74082FF582E43480E0
:08183600F583EEF00FBF06CAB6
:01183E002287
:10183F00E4FF74092FF582E43429F583E0FEE42FE9
:10184F00F582E43480F583EEF0300918740F2FF52C
:10185F0082E43429F583E0FE74082FF582E43480A6
:08186F00F583EEF00FBF06CA7D
:01187700224E
:101B1500E4FF74092FF582E43429F58374FFF0306E
:101B2500090D740F2FF582E43429F58374FFF00F46
:031B3500BF06DF09
:011B3800228A
:0800030090E600E054E7F02252
:101630007AE779407F40AB077D017F037E0012157A
:101640009D90E740E064D06005E0900EC2F090E726
:1016500040E024FD600F0470147BFF7A1B797F1239
:1016600014ECC209227BFF7A1B798A80067BFF7A01
:091670001B79951214ECD2092239
:081DB30090E600E054E7F02285
:01002A0022B3
:01004A002293
:10073C00D2071209F150030208C890E6B9E024ED83
:10074C00700302082A24E37003020839241E600394
:10075C000208C690E6BEE090E68BF090E6A0E020A2
:10076C00E1F93009047F0C80027F068F2990E6BDE9
:10077C00E0FF90E6BCE04F7033300921744125292D
:10078C00F582E434E7F583E0F4540FFF90E6BAE029
:10079C005401FEC454F04F9028FAF0F590744025A3
:1007AC0029F582E434E7F583E0F480607440252970
:1007BC00300942F582E434E7F583E0F4FF74422516
:1007CC0029F582E434E7F583E04F9028F9F0F580C1
:1007DC0074412529F582E434E7F583E0F4FF744392
:1007EC002529F582E434E7F583E04F540F9028FA7D
:1007FC00F0F590801DF582E434E7F583E0F4FF74A6
:10080C00412529F582E434E7F583E04F9028F9F08F
:10081C00F5807B017AE779401214360208C8E5802E
:10082C00F490E740F0E590F4541FA3807DE4F529A3
:10083C0074FB2529F582E43428F583E0FF74402508
:10084C0029F582E434E7F583EFF030091A740125B9
:10085C0029F582E43429F583E0FF74462529F582D5
:10086C00E434E7F583EFF00529E529B406C29028B6
:10087C00F9E0F4FFA209E4FC33FD90E74675F006BD
:10088C00120D6DEC75F006A42583F583EFF090281E
:10089C00FAE0F4541FFF90E74775F006ED120D6D6A
:1008AC00EC75F006A42583F583EFF0E490E68AF06E
:0D08BC0090E6BEE090E68BF08002D322C3F0
:0108C900220C
:041DDF000000000000
:101D6200021D1DDF02080000011001010C01010A21
:011D7200016F
:101D2B0090289FE0700690289EE060030200361218
:031D3B00002E2255
:101BA0007E007F797D007B017A28799C120D9F90C1
:101BB000289C7409F0E4A3F0121AC5121491021CB7
:011BC000D450
:10000E007D0212159590289CE0B40904A3E06003CC
:0C001E00021BA07D79121595121491228E
:101CD4007A287B9C7D797F017E1F120DCB7D797FD5
:061CE400007E1F021DE757
:10129E00121D2B90E6BEE0F535753702E535605729
:1012AE00C3944050058535368003753640E490E68C
:1012BE008AF090E68BE536F090E6A0E020E1F9E4C6
:1012CE00F534E534C39536502574402534F582E463
:1012DE0034E7F583E0FFAE370537EE7C007B012463
:1012EE009CF9EC3428FAEF120D39053480D4C3E59D
:0A12FE00359536F53580A5021D2B4D
:0F1D8400D3E546950EE545950D4003121D9322BC
:01005200228B
:101B39009028A1E0FE9028A0E07C002400F50EEC9E
:101B49003EF50D450E7007C28CC2A9C20822D28C7F
:031B5900D2A922EC
:011DF70022C9
:1017070090E6BEE090E68BF090E6A0E020E1F9E4F9
:10171700FF74422FF582E434E7F583E0FEEF7C00A7
:101727007B012407F9EC3429FAEE120D390FBF0EAD
:10173700E090E740E09028A0F090E741E09028A1F2
:04174700F0021B3958
:0B1D930012183FE4F545F546D2082287
:101C8C00E4F545F546C28CC2A9538EF75389F1434E
:081C9C008901121DF7021B393A
:1019B400E50945086017E50915097002150814C3FF
:1019C40094FFE50864809480501602004E3007109E
:1019D4007508057509FF120046C207E4F545F5468A
:0119E40022E0
:1008CA0090E6B8E020E70302097FE4F5339028A018
:1008DA00E0FFAE33053374402EF582E434E7F58346
:1008EA00EFF09028A1E0FFAE33053374402EF58275
:1008FA00E434E7F583EFF0E4F532E532C3940E50C1
:10090A00247E007B0174072532F9EE3429FA120C91
:10091A00F3FF74402533F582E434E7F583EFF005FD
:10092A0032053380D5AE33053374402EF582E43474
:10093A00E7F583E546F0E545FFAE33053374402E0F
:10094A00F582E434E7F583EFF0A208E433FFAE332F
:10095A00053374402EF582E434E7F583EFF0C208DC
:10096A00E490E68AF090E6BEE090E68BF090E6A08E
:10097A00E04480F02290E6BEE090E68BF090E6A09C
:10098A00E020E1F990E6BEE0640E705AE4F533AF78
:10099A0033053374402FF582E434E7F583E0902879
:1009AA00A0F0AF33053374402FF582E434E7F583C2
:1009BA00E09028A1F0E4F532E532C3940E50247495
:1009CA00402533F582E434E7F583E0FFE5327C0025
:1009DA007B012407F9EC3429FAEF120D39053205A7
:0609EA003380D5121B3919
:0109F00022E4
:041DD7007510012260
:10130800121D2B90E6BEE0F535E4F537E53560575C
:10131800C3944050058535368003753640E490E621
:101328008AF090E68BE536F090E6A0E020E1F9E45B
:10133800F534E534C39536502574402534F582E4F8
:1013480034E7F583E0FFAE370537EE7C007B0124F8
:10135800B7F9EC3428FAEF120D39053480D4C3E517
:07136800359536F53580A52F
:01136F00225B
:101543001510E510704B9028B7E0F5101217CDE495
:10155300F5229028F8E0FFE522C39F5031E52225CC
:10156300E024B8F582E43428F583E0F523E5222569
:10157300E024B9F582E43428F583E0F524547FFDB3
:10158300E524339204AF231211A5052280C4121857
:011593000651
:011594002234
:101BC10090E6BEE090E68BF090E6A0E020E1F9908F
:101BD100E740E09028A2F090E741E09028A3F022AE
:10111A00150CE50C60030211A49028A2E0F50C7BE3
:10112A00017A297915121225E4FFFE74152EF5822B
:10113A00E43429F583E0FD74002EF582E43428F5C1
:10114A0083E06DF97D01E4FCECC394085046E95D47
:10115A006029740C2FF582E43428F583E014F074C6
:10116A000C2FF582E43428F583E0702074002EF504
:10117A0082E43428F583E06DF080009028A3E0FB38
:10118A00740C2FF582E43428F583EBF00CED25E09E
:0A119A00FD0F80B40EEE640C70919E
:0111A4002228
:101CA40090E6BEE090E68BF090E6A0E020E1F990AB
:081CB400E740E09028A4F022B3
:101A4100E4FF746C2FF582E43428F583E4F07484A8
:101A51002FF582E43428F58374FFF074782FF58232
:0B1A6100E43428F583E4F00FBF0CD73D
:011A6C002257
:1013D400150AE50A705B9028A4E0F50A7B017A28D7
:1013E400796C121225E4FF74842FF582E43428F515
:1013F40083C083C082E0FE746C2FF582E43428F548
:1014040083E0FDEE5DD082D083F074782FF582E422
:101414003428F583C083C082E0FE746C2FF582E427
:101424003428F583E0FDEE4DD082D083F00FBF0C5D
:01143400B601
:011435002294
:041DDB00750F01225D
:100F6C00150FE50F603DE4F5229028B6E0FFE52271
:100F7C00C39F507C74152522F8E6602316E6701F7B
:100F8C00E52225E024A6F582E43428F583E0FE541E
:100F9C007FFFEE30E7047D0080027D0112174B05C8
:100FAC002280C69028A5E0F50FE4F5229028B6E043
:100FBC00FFE522C39F5039E52225E024A7F582E402
:100FCC003428F583E0FF74152522F8A607E52225C1
:100FDC00E024A6F582E43428F583E0FE547FFFEE8E
:100FEC0030E7047D0180027D0012174B052280BC86
:010FFC0022D2
:1019500090E6BEE090E68BF090E6A0E020E1F9E4AE
:10196000FF74402FF582E434E7F583E0FEEF7C005E
:101970007B0124A5F9EC3428FAEE120D390FBF12C1
:01198000E086
:011981002243
:10005600E4F53390E6B8E030E77790E6BEE0FF706F
:100066000490E68BF0BF010D90E7407479F090E6BE
:100076008B7401F01FEF605190E6A0E020E1F9EFEC
:10008600C3944050048F328003753240E4FEEEC3C1
:1000960095325023AD3305337C007B01749C2DF9DA
:1000A600EC3428FA120CF3FD74402EF582E434E7A2
:1000B600F583EDF00E80D7E490E68AF090E68BE5C6
:1000C60032F0C3EF9532FF80AC90E6A0E04480F0BA
:1000D6002290E6BFE0FF90E6BEE04F707790E6BD67
:1000E600E0704D90E6BCE024EF6023249F6030244E
:1000F600FD603324F360342472703590E6BAE06410
:10010600CE702DA3E064AC7027121CD4802290E63A
:10011600BAE0B4CE1BA3E0B4AC16121BA08011E467
:100126009028B6F0800A750F018005E49028F8F053
:1001360090E6BDE06480600302037890E6BCE0646C
:1001460001600302037890E6BAE090289EF090E6FC
:10015600BB02020B90E6BFE0600302037890E6BDA7
:10016600E0FE90E6BCE07C002400FFEC3EFE60036F
:10017600020378EF120D7901B12001B12101B122FC
:1001860001B12301E62F021341022151022F53022E
:100196004F61025D63027D71028B7302AB740300D3
:1001A60081030B830328840000037890E6BEE0B445
:1001B600770312129E90E6BCE030E0031214919091
:1001C600E6BCE020E10302037890E6BAE064CE6084
:1001D60003020378A3E064AC6003020378021CD434
:1001E60090E6BEE064026003020378E090E68BF0DE
:1001F60090E6A0E020E1F9121D2B90E740E0902860
:100206009EF090E741E090289FF0021D2B90E6BEFD
:10021600E06410600302037802170790E6BEE0640C
:10022600026003020378021BC190E6BEE06401602F
:1002360003020378E090E68BF090E6A0E020E1F977
:1002460090E740E09028A2F02290E6BEE0640160CC
:1002560003020378021CA490E6BEE0640160030278
:100266000378E090E68BF090E6A0E020E1F990E7D5
:1002760040E09028A4F02290E6BEE06412600302FB
:10028600037802195090E6BEE06401600302037829
:10029600E090E68BF090E6A0E020E1F990E740E000
:1002A6009028A5F02290E6BEE0640260030203787F
:1002B6009028B6E0C39408400302037890E6BEE0B7
:1002C60090E68BF090E6A0E020E1F990E740E0FFB1
:1002D6009028B6E0FE25E024A4F582E43428F583D0
:1002E600EFF090E741E0FFEE25E024A5F582E43447
:1002F60028F583EFF09028B6807590E6BEE064425C
:10030600707002130890E6BEE064017065E090E646
:100316008BF090E6A0E020E1F990E740E09028B766
:10032600F02290E6BEE0640270489028F8E0C3949C
:1003360020503F90E6BEE090E68BF090E6A0E020ED
:10034600E1F990E740E0FF9028F8E0FE25E024B6CA
:10035600F582E43428F583EFF090E741E0FFEE25DF
:10036600E024B7F582E43428F583EFF09028F8E02E
:0203760004F091
:010378002262
:101C560090E6047480F00000007402F00000007446
:0B1C660006F0000000E4F00000002287
:011DF80022C8
:10178E00E4F5297AE779407F40AB077D087FF87E44
:10179E001D12159DE4F52974402529F582E434E7E0
:1017AE00F583E0FDE52975F002A42416F9740F35D2
:0E17BE00F08982F583EDF00529E529B408D9FC
:0117CC0022FA
:1016790090E678E05410FFC4540F4450F51113E478
:1016890033F51390E600E054E74410F0438E20123E
:10169900002E120003121DCB12178E121630D20023
:1016A90012000E121DD7121C8C121A41121DDB12C8
:0816B9001D2B12004E021DB3AF
:101C000012002A1219B4121D84E5B190E68020E773
:0E1C100006E04408F08004E054F7F002004AB9
:0614EC008B298A2A892BDE
:1014F200E4F52C121D168F2DE52D25E02402900F08
:101502004CF0E4F52CAF2DEF3395E0FEC3E52C9FB4
:10151200EE6480F87480985027AB29AA2AA92B85FB
:101522002C82758300120D0CFDE52C75F002A424AB
:101532004EF9740F35F08982F583EDF0052C80C5E4
:011542002286
:0615E5008E408F41AC05B1
:1015EB00E4FDE5136012E540FF7E000DEE251EF5D0
:1015FB0082E4351DF583EFF0AE050DE51E2EF58269
:10160B00E4351DF583E541F0AF050DE51E2FF582A1
:10161B00E4351DF583ECF0AB1EAA1DAF11121C3A7D
:05162B00AF110218E6FA
:031DE7000215E5FD
:0A0DCB008E3A8F3B8D3C8A3D8B3E33
:100DD500E4F53FE53FC3953C5020053BE53BAE3A86
:100DE5007002053A14FFE53E253FF582E4353DF5F1
:0A0DF50083E0FD121DE7053F80D9E1
:010DFF0022D1
:081595007A287B9C7F017E1F78
:0A159D008E3A8F3B8D3C8A3D8B3E59
:1015A700E4FDF53FE5136012E53AFF7E000DEE25F9
:1015B7001EF582E4351DF583EFF0AE050DE51E2E11
:1015C700F582E4351DF583E53BF0AB1EAA1DAF118F
:0E15D700121C3AAB3EAA3DAD3CAF11021C1EE9
:10059E0090E6BAE0753200F533A3E0FEEE423290FB
:1005AE00E6BEE0753400F535A3E0FEEE423490E68B
:1005BE00B8E064C060030206A9E535453470030255
:1005CE00073B90E6A0E020E1F9C3E5359440E53421
:1005DE00940050088534368535378006753600759B
:1005EE00374090E6B9E064A3705790E6BCE0B401E2
:1005FE001BA3E0701790E6BBE030E71090E7407465
:10060E0003F0A37401F0A37403F0806AE4F538F5E7
:10061E0039C3E5399537E5389536505AE5332539DE
:10062E00F582E5323538F583E0FF74402539F582E1
:10063E00E434E7F583EFF00539E53970D4053880F9
:10064E00D0E4F538F539C3E5399537E538953650A8
:10065E001874402539F582E434E7F58374CDF0053E
:10066E0039E53970E1053880DDAD377AE77B40AF8B
:10067E0033AE3212159DE490E68AF090E68BE537A4
:10068E00F02533F533E5363532F532C3E53595379A
:10069E00F535E5349536F5340205C790E6B8E064D5
:1006AE0040600302073BE5354534700302073BE427
:1006BE0090E68AF090E68BF090E6A0E020E1F990CB
:1006CE00E68BE0753600F53790E6B9E0B4A335E475
:1006DE00F538F539C3E5399537E538953650327426
:1006EE00402539F582E434E7F583E0FFE53325391B
:1006FE00F582E5323538F583EFF00539E53970D4FA
:10070E00053880D0AD377AE77B40AF33AE32120D6D
:10071E00CBE5372533F533E5363532F532C3E535DE
:0D072E009537F535E5349536F5340206B4FF
:01073B00229B
:100C1400E4FF90E6B8E020E703020CF20F0F744003
:100C24002401F582E434E7F5837409F00F74402459
:100C340002F582E434E7F583E4F00F74402403F50D
:100C440082E434E7F583E4F00F74402404F582E48D
:100C540034E7F5837402F00F74402405F582E4341C
:100C6400E7F583740CF00F74402406F582E434E74E
:100C7400F583E4F00F74402407F582E434E7F58348
:100C8400E4F00F74402408F582E434E7F58374FF3C
:100C9400F00F74402409F582E434E7F58374FFF01F
:100CA4000F7440240AF582E434E7F5837408F00FE6
:100CB4007440240BF582E434E7F5837420F00F7458
:100CC40040240CF582E434E7F583745FF00F74403C
:100CD400240DF582E434E7F583745FF090E740EF88
:0E0CE400F0E490E68AF090E6BEE090E68BF039
:010CF20022DF
:0B1D9E00E50E450D7003D38001C32249
:021DED00D322FF
:021DEF00D322FD
:081DBB0090E6BAE0F50BD3221B
:101D3E0090E740E50BF0E490E68AF090E68B04F035
:021D4E00D3229E
:081DC30090E6BAE0F512D3220C
:101D500090E740E512F0E490E68AF090E68B04F01C
:021D6000D3228C
:021DF100D322FB
:021DF300D322F9
:021DF500D322F7
:1009F10090E6B9E0120D790A2F100A2F110A5D1441
:100A01000ACE150A1D2E0A173C0A293F0A23A20AFB
:100A110023A300000B08120056020B0A1208CA0297
:100A21000B0A12059E020B0A120C14020B0A90E625
:100A3100B8E030E70C7B017AE77940121225020A0F
:100A4100F290E6BEE090E68BF090E6A0E020E1F9BE
:100A51007B017AE77940121436020B0AE4F52B7414
:100A61006C252BF582E43428F583E0FF7440252BB7
:100A7100F582E434E7F583EFF0052BE52BB40CDFC9
:100A8100E4F52B7484252BF582E43428F583E0FF0B
:100A9100744C252BF582E434E7F583EFF0052BE563
:100AA1002BB40CDFE4F52B7478252BF582E4342884
:100AB100F583E0FF7458252BF582E434E7F583EFE5
:100AC100F0052BE52BB40CDF121A418024E4F52B41
:100AD1007400252BF582E43428F583E0FF7440256A
:100AE1002BF582E434E7F583EFF0052BE52BB40C0D
:100AF100DFE490E68AF090E6BEE090E68BF090E6C7
:0A0B0100A0E04480F08002C322D37C
:010B0B0022C7
:101BE100C0E0C083C08290E6B5E04401F0D2015369
:0F1BF10091EF90E65D7401F0D082D083D0E032A6
:101CEA00C0E0C083C0825391EF90E65D7404F0D0E7
:061CFA0082D083D0E0322D
:101D0000C0E0C083C0825391EF90E65D7402F0D0D2
:061D100082D083D0E03216
:10187800C0E0C083C08290E680E030E70E8543492F
:1018880085444A854D4B854E4C800C854D49854E87
:101898004A85434B85444C5391EF90E65D7410F0B4
:0718A800D082D083D0E032B2
:101CBC00C0E0C083C082D2035391EF90E65D7408FC
:081CCC00F0D082D083D0E03299
:1018AF00C0E0C083C08290E680E030E70E854349F8
:1018BF0085444A854D4B854E4C800C854D49854E50
:1018CF004A85434B85444C5391EF90E65D7420F06D
:0718DF00D082D083D0E0327B
:011DF90032B7
:011DFA0032B6
:011DFB0032B5
:011DFC0032B4
:011DFD0032B3
:011DFE0032B2
:011DFF0032B1
:011E000032AF
:011E010032AE
:011E020032AD
:011E030032AC
:011E040032AB
:011E050032AA
:011E060032A9
:011E070032A8
:011E080032A7
:011E090032A6
:011E0A0032A5
:011E0B0032A4
:011E0C0032A3
:011E0D0032A2
:011E0E0032A1
:011E0F0032A0
:011E1000329F
:011E1100329E
:011E1200329D
:011E1300329C
:011E1400329B
:011E1500329A
:011E16003299
:011E17003298
:011E18003297
:011E19003296
:011E1A003295
:011E1B003294
:011E1C003293
:0A1DA9000001020203030404050513
:03000B00021C7163
:101C7100C0E0C0D00542E542B43C0B0546E54670E4
:0B1C8100020545754200D0D0D0E032D3
:100FFD00E4F528F527F526F525C203C200C202C285
:10100D000112167975470E7548B8754F0E7550CA91
:10101D0075430E7544D4754D0E754EF475510F759F
:10102D005214D2E843D82090E668E04409F090E6E7
:10103D005CE0443DF0D2AFD2061219E590E680E0B7
:10104D0054F7F0538EF8C203300105120379C20133
:10105D00300329121D9E5024C203121AF0200016CF
:10106D0090E682E030E704E020E1EF90E682E030A8
:10107D00E604E020E0E4121A6D121DED121C008052
:01108D00C79B
:1003790090E6B9E0700302042A1470030204A7246A
:10038900FE700302052A24FB70030204241470037F
:1003990002041E1460731460762405600302058A42
:1003A900121DEF400302059690E6BBE024FE602291
:1003B90014603324FD601114602224067048E54757
:1003C90090E6B3F0E5488037E54F90E6B3F0E550A5
:1003D900802DE54990E6B3F0E54A8023E54B90E6A8
:1003E900B3F0E54C801990E6BAE0FF121A99AA0613
:1003F900A9077B01EA494B600DEE90E6B3F0EF9057
:10040900E6B4F002059602058F121D5002059612F8
:100419001DC3020596121DBB020596121D3E02055B
:1004290096121DF1400302059690E6B8E0247F601C
:100439001514601924027063A200E43325E0FFA2B9
:1004490002E4334F8041E490E740F0803F90E6BCFE
:10045900E0547EFF7E00E0D394807C0040047D015F
:1004690080027D00EC4EFEED4F24A9F582741D3EFD
:10047900F583E493FF3395E0FEEF24A1FFEE34E624
:100489008F82F583E0540190E740F0E4A3F090E611
:100499008AF090E68B7402F002059602058F121D10
:1004A900F3400302059690E6B8E024FE60162402A4
:1004B900600302059690E6BAE0B40105C2000205A0
:1004C9009602058F90E6BAE0705590E6BCE0547E3E
:1004D900FF7E00E0D394807C0040047D0180027D92
:1004E90000EC4EFEED4F24A9F582741D3EF583E420
:1004F90093FF3395E0FEEF24A1FFEE34E68F82F5FA
:1005090083E054FEF090E6BCE05480131313541FAB
:10051900FFE0540F2F90E683F0E04420F0806E80D6
:1005290065121DF5506790E6B8E024FE601A2402B2
:10053900705B90E6BAE0B40104D200805090E6BA4C
:10054900E0B402028047803E90E6BCE0547EFF7E24
:1005590000E0D394807C0040047D0180027D00ECA2
:100569004EFEED4F24A9F582741D3EF583E493FFF9
:100579003395E0FEEF24A1FFEE34E68F82F5838008
:100589000812073C500790E6A0E04401F090E6A06D
:04059900E04480F0CA
:01059D00223B
:03003300021DE3C8
:041DE30053D8EF32B0
:101B5C00902921EFF0F5CB8FCDAF05A3EFF0F5CAAF
:101B6C008FCCE4F5C8758E19D2BDD2AFD2ADD2CA26
:031B7C00F55922F6
:0D00360090289FE0FF90289EE0FD021B5CDB
:031DEA00AF5922CC
:101D7400AD07AC06C3E49DFBE49CFFEBFD021B5CDA
:05002E00C2CAC2AD22B0
:03002B000213704D
:10137000C0E0C0F0C083C082C0D075D000C000C043
:1013800001C002C003C004C005C006C0079028A267
:10139000E0600312111A9028A4E060031213D490A5
:1013A00028B6E06003120F6C9028F8E060099028DE
:1013B000B7E06003121543C2CFD007D006D005D0E6
:1013C00004D003D002D001D000D0D0D082D083D0BE
:0413D000F0D0E03247
:03004300020E00AA
:03005300020E009A
:100E0000021BE100021D0000021CEA00021CBC00E3
:100E1000021878000218AF00021DF900021DFA0046
:100E2000021DFB00021DFC00021DFD00021DFE0054
:100E3000021DFF00021E0000021E0100021E020031
:100E4000021E0300021DFA00021E0400021E05001D
:100E5000021E0600021E0700021E0800021E0900F4
:100E6000021E0A00021DFA00021DFA00021DFA000D
:100E7000021E0B00021E0C00021E0D00021E0E00C0
:100E8000021E0F00021E1000021E1100021E1200A0
:100E9000021E1300021E1400021E1500021E160080
:100EA000021E1700021E1800021E1900021E1A0060
:080EB000021E1B00021E1C00C3
:101A6D0090E682E030E004E020E60B90E682E03084
:101A7D00E119E030E71590E680E04401F07F147E37
:0C1A8D00001216C190E680E054FEF0222A
:101AF00090E682E044C0F090E681F0438701000068
:041B000000000022BF
:1019E50030060990E680E0440AF0800790E680E042
:1019F5004408F07FDC7E051216C190E65D74FFF0A9
:0F1A050090E65FF05391EF90E680E054F7F02207
:081DCB00E4F558D2E9D2AF2281
:1018E60090E678E020E6F9C2E990E678E04480F0F8
:1018F600EF25E090E679F090E678E030E0F990E6C2
:1019060078E04440F090E678E020E6F990E678E06A
:0619160030E1D6D2E92207
:10198200A90790E678E020E6F9E558702390E6781A
:10199200E04480F0E925E090E679F08D53AF03A9A9
:1019A200077554018A558956E4F557755801D322B3
:0219B200C3224E
:10191C00A90790E678E020E6F9E558702590E6787E
:10192C00E04480F0E925E0440190E679F08D53AF76
:10193C0003A9077554018A558956E4F55775580360
:04194C00D322C322BD
:03004B00020B0C99
:100B0C00C0E0C083C082C085C084C086758600C02A
:100B1C00D075D000C000C001C002C003C006C00721
:100B2C0090E678E030E206755806020BF690E6780F
:100B3C00E020E10CE55864026006755807020BF6DC
:100B4C00E55824FE605F14603624FE7003020BE748
:100B5C0024FC7003020BF324086003020BF6AB5465
:100B6C00AA55A956AF5705578F82758300120D0CE5
:100B7C0090E679F0E55765537070755805806B9069
:100B8C00E679E0AB54AA55A956AE578E8275830010
:100B9C00120D4B755802E5536401704E90E678E0E7
:100BAC004420F08045E55324FEB5570790E678E0E5
:100BBC004420F0E55314B5570A90E678E04440F031
:100BCC0075580090E679E0AB54AA55A956AE578EED
:100BDC0082758300120D4B0557800F90E678E04428
:100BEC0040F075580080037558005391DFD007D042
:100BFC0006D003D002D001D000D0D0D086D084D083
:080C0C0085D082D083D0E032D4
:021A9900A9079B
:101A9B00AE51AF528F828E83A3E064037017AD01FA
:101AAB0019ED7001228F828E83E07C002FFDEC3EBE
:091ABB00FEAF0580DF7E007F0014
:011AC40022FF
:101C1E0012191CE55824FA600E146006240770F39E
:0C1C2E00D322E4F558D322E4F558D32269
:101C3A00121982E55824FA600E146006240770F31C
:0C1C4A00D322E4F558D322E4F558D3224D
:1016C1008E298F2A90E600E054187012E52A240131
:1016D100FFE43529C313F529EF13F52A801590E6A8
:1016E10000E05418FFBF100BE52A25E0F52AE52993
:1016F10033F529E52A152AAE29700215294E600510
:06170100121B0480EE2221
:101B04007400F58690FDA57C05A3E582458370F9F4
:011B140022AE
:0300000002108E5D
:0C108E00787FE4F6D8FD75815A0210D579
:100CF300BB010689828A83E0225002E722BBFE02FF
:090D0300E32289828A83E4932231
:100D0C00BB010CE58229F582E5833AF583E022509C
:100D1C0006E92582F8E622BBFE06E92582F8E222E6
:0D0D2C00E58229F582E5833AF583E4932200
:100D3900BB010689828A83F0225002F722BBFE0199
:020D4900F32293
:100D4B00F8BB010DE58229F582E5833AF583E8F0DE
:100D5B00225006E92582C8F622BBFE05E92582C88A
:020D6B00F22272
:0C0D6D00A42582F582E5F03583F5832291
:100D7900D083D082F8E4937012740193700DA3A309
:100D890093F8740193F5828883E47374029368601D
:060D9900EFA3A3A380DF1D
:101D1600E4FFFE120CF3600C0FEF70010E09E97080
:051D2600F20A80EF222B
:100D9F00EF4E6012EF60010EEDBB010B89828A836B
:100DAF00F0A3DFFCDEFA2289F05007F709DFFCA978
:0C0DBF00F022BBFEFCF309DFFCA9F022CF
:10109A00020FFDE493A3F8E493A34003F68001F260
:1010AA0008DFF48029E493A3F85407240CC8C33357
:1010BA00C4540F4420C8834004F456800146F6DF26
:1010CA00E4800B0102040810204080901D62E47E37
:1010DA00019360BCA3FF543F30E509541FFEE4931B
:1010EA00A360010ECF54C025E060A840B8E493A3E2
:1010FA00FAE493A3F8E493A3C8C582C8CAC583CA0D
:10110A00F0A3C8C582C8CAC583CADFE9DEE780BEC4
:011D7300006F
:00000001FF
